:020000040000FA
:100000008316051085100511851205169F019F1591
:100010001F139F121F1683128B130730990085162A
:100020000510851005116B2005156B2085146B20BC
:1000300005146B201F141F159F151F139F134720B6
:1000400003141E08CC3C0515031C05111E08993C21
:100050008514031C85101E08663C0514031C05103E
:10006000051D3828851C3D28051C422885161F289B
:1000700085125020851662201F288512592085166A
:1000800059201F2885126220851650201F28033012
:10009000A000A00B49289F149F184C280C1308009F
:1000A0007D30A0000730A100A00B5428A10B5428DC
:1000B0000800EE30A0004130A100A00B5D28A10B8C
:1000C0005D2808005F30A0007C30A100A00B6628EE
:1000D000A10B66280800AD30A0001330A100063047
:1000E000A200A00B7128A10B7128A20B7128080097
:02400E00F43F7D
:00000001FF
